:060000000200E6020F4CB5
:03000B00020DA93A
:0300130002137A5B
:01001B0032B2
:0300230002140BB9
:01002B0032A2
:0300330002066C56
:03003B0002155556
:01004300328A
:01004B003282
:01005300327A
:01005B003272
:01006300326A
:03006B0002073554
:0300730002074D34
:03007B0002076316
:03008300020779F8
:03008B000207ADBC
:030093000207AEB3
:03009B000207C693
:0300A3000207C78A
:0300AB000207C881
:0300B300020A9CA2
:0300BB00020BE94C
:0300C300020BFF2E
:0100CB003202
:0100D30032FA
:0300DB00020C4BC9
:0300E300020C61AB
:030164000201672E
:0501670012016C80FE96
:05016C00C203C201C244
:0401710002C20012B4
:040175000670750893
:030179007775098E
:03017C0016750AEB
:03017F0089750B74
:0301820016750CE3
:03018500C5750D30
:04018800167A7774F8
:09018C0016FB54E0700302025559
:0401950075127775F3
:0301990013167CBE
:04019C00DD7D167E71
:0A01A000777F16ECC39EFCED9FFD77
:0A01AA0074022CFCE43DFD8C0E8D68
:0501B4000F751000753D
:0A01B9001100780079007A007B0045
:0901C300C3E8950EE9950FEA95D9
:0A01CC0010EB9511501B748028F50C
:0E01D60082E439F58374CDF008B800E109B970
:0901E40000DD0ABA00D90B80D637
:0801ED007A007B007800790024
:0901F500C3EA950EEB950FE895A5
:0A01FE0010E99511502974802AFCC5
:0A020800E43BFDAE12AF13EA2EF541
:0E02120082EB3FF583E0FE8C828D83F00ABA0A
:0D02200000D30BBB00CF08B800CB0980C88D
:07022D00750880E4F5097A71
:0A023400777B16EA2480FAEB34FF12
:08023E00FBE50AC39AF50AE58D
:050246000B9BF50BE528
:06024B000CC39AF50CE55E
:040251000D9BF50DFF
:0E025500D2E843D820907FAFE0FA4401F09049
:0C0263007FAEE0FA441DF0D2AFD20412CE
:05026F001744538EF856
:070274003000051202A1C2D7
:01027B000082
:09027C0030031D1206E55018C202
:010285000375
:0702860012192B2001089062
:07028D007FD6E0FA20E7F242
:080294001219691206E9E433B6
:05029C001206CA80D328
:0C02A100907FE9E0FA24F4500302064CC0
:0702AD00EA2A2A9002B47353
:0702B40002046E02052002A6
:0602BB00064C0205C8021A
:0602C100064C02064C028F
:0602C70002D802064C0201
:0602CD00046602045E025B
:0502D300044E02045678
:0802D8001206ED400302065E70
:0A02E000907FEBE0FABA0102800DF6
:0502EA00BA0202801AB7
:0502EF00BA0302805378
:0302F40002043EC3
:0702F700907FD4E509F0AA95
:0902FE00087B00907FD5EAF002B4
:02030700065E90
:0E030900907FEAE0FAF582121795AA82AB8384
:0E0317007C008A058B068C07EA4B4C60138D28
:0E032500028E03907FD4EBF07B00907FD5EA30
:04033300F002065E70
:0E033700907FB4E0FA430201907FB4EAF00236
:02034500065E52
:0E034700907FEAE0FAF5821218F0AA82AB83EA
:0E0355007C008A058B068C07EA4B4C70030275
:02036300042E66
:050365008D188E198FB8
:0C036A001A8D828E838FF0121988FF908C
:0D0376007FEEE0FEC39F5005907FEEE0FF9C
:06038300EF7003020420EC
:03038900BF400072
:09038C00E433FEE4F514F515F567
:0303950016F51743
:07039800EE60048F038002F8
:02039F007B40A1
:0B03A1007C007D007A00C3E5149BE5A2
:0603AC00159CE5169DE51D
:0703B200179A5033E51424F3
:0503B90000FAE5153417
:0503BE007FFBAC18AD4F
:0703C30019E5142CF582E599
:0C03CA00153DF583E0FC8A828B83F00572
:0603D60014E4B5140C054F
:0503DC0015B515070531
:0503E10016B516B3057E
:0103E60017FF
:0203E70080AFE5
:0303E900BF400012
:0603EC0050048F028002A4
:0203F2007A404F
:0803F400907FB5EAF0BF400064
:0603FC0050048F02800294
:020402007A403E
:0A040400EFC39AFF74402518F518A5
:05040E00E43519F519A9
:0B041300907FB4E0FA20E203020383B4
:02041E0080F369
:0C042000907FB5E4F0907FB47402F0020D
:02042C00065E6A
:0E042E00907FB4E0FA430201907FB4EAF0023E
:02043C00065E5A
:0E043E00907FB4E0FA430201907FB4EAF0022E
:02044C00065E4A
:08044E00120715E43302065EFB
:0804560012070BE43302065EFD
:08045E001206F1E43302065E10
:080466001206FBE43302065EFE
:08046E00120725400302065E9F
:0A047600907FE8E0FABA8002800DE2
:05048000BA8102802991
:05048500BA820280367E
:03048A0002051058
:0A048D00E4A2013325E0FAE4A20224
:0E04970033FB4202907F00EAF0907F01E4F018
:0904A500907FB57402F002065EBE
:0A04AE00907F00E4F0907F01F090D1
:0804B8007FB57402F002065E3C
:0E04C000907FECE0FA7B00F4FAEBF4FB5302C1
:0E04CE0080E4FBC4CAC4540F6ACA540FCA6A41
:0604DC00CA30E30244F007
:0E04E200FB907FECE0FB74075B2A25E0FA2418
:0A04F000B4F582E4347FF583E0FAEE
:0E04FA00530201907F00EAF0907F01E4F09041
:080508007FB57402F002065EEB
:0E051000907FB4E0FA430201907FB4EAF0025B
:02051E00065E77
:08052000120729400302065EE8
:0C052800907FE8E0FA6008BA0202802030
:0305340002065E5E
:0B053700907FEAE0FABA0105C2010261
:02054200065E53
:0E054400907FB4E0FA430201907FB4EAF00227
:02055200065E43
:0E055400907FEAE0705E907FECE0FA7B00F4AE
:0E056200FAEBF4FB530280E4FBC4CAC4540F4E
:0C0570006ACA540FCA6ACA30E30244F0A1
:0E057C00FB907FECE0FB74075B2A25E0FA247D
:0A058A00B4F582E4347FF583E4F059
:0D059400907FECE05480FAC423541FFA90CD
:0D05A1007FECE0FB74075B907FD72AF090A1
:0A05AE007FD7E0FA4420F002065E59
:0E05B800907FB4E0FA430201907FB4EAF002B3
:0205C600065ECF
:0805C80012072D400302065E3C
:0C05D000907FE8E0FA6008BA0202801E8A
:0305DC0002065EB6
:0C05DF00907FEAE0FABA0104D2018073B8
:0E05EB00907FB4E0FA430201907FB4EAF08002
:0105F900649D
:0E05FA00907FEAE0703D907FECE0FA7B00F429
:0E060800FAEBF4FB530280E4FBC4CAC4540FA7
:0C0616006ACA540FCA6ACA30E30244F0FA
:0E062200FB907FECE0FB74075B2A25E0FA24D6
:0A063000B4F582E4347FF583740111
:03063A00F080212C
:0E063D00907FB4E0FA430201907FB4EAF080AF
:01064B00129C
:0E064C00120731500D907FB4E0FA4302019086
:04065A007FB4EAF08F
:0E065E00907FB4E0FA430202907FB4EAF022EB
:04066C0053D8EF323E
:0E067000907FDEE0FA4416F0907FDFE0FA445F
:0E067E0016F0907FDDE4F0E0FA907FDD740965
:0E068C004AF0907FDDE0FA4412F0907FAD74EA
:0E069A0016F0907FAC7416F0907FC7E4F090DD
:0806A8007FC9F0907FCDF075D1
:0906B0001D01907F9C74FFF01203
:0606B9000D0F120E8C1261
:0606BF001657120D8A120D
:0506C50012C0D2012269
:0406CA007A307B7592
:0506CE001ABAFF011B38
:0806D300EA4B70F77A307B75E9
:0506DB001ABAFF011B2B
:0506E000EA4B70F72257
:0406E50075820122F7
:0406E90075820122F3
:0406ED0075820122EF
:0A06F100907FEAE0F51B75820122FC
:0706FB00907F00E51BF09069
:090702007FB57401F0758201223B
:0A070B00907FEAE0F51C75820122E0
:07071500907F00E51CF0904D
:09071C007FB57401F07582012221
:0407250075820122B6
:0407290075820122B2
:04072D0075820122AE
:0407310075820122AA
:0C073500C0E0C082C083D2005391EF905E
:0C0741007FAB7401F0D083D082D0E03296
:0E074D00C0E0C082C0835391EF907FAB740474
:08075B00F0D083D082D0E0321F
:0E076300C0E0C082C0835391EF907FAB740260
:08077100F0D083D082D0E03209
:0E077900C0E0C082C083907FC7E4F0907FC9CB
:0A078700F0907FCBF0907FCDF09052
:090791007FCFE4F0907FD1F090DD
:0E079A007FD3F05391EF907FAB7410F0D083BB
:0507A800D082D0E03218
:0107AD003219
:0C07AE00C0E0C082C083D2035391EF90E2
:0C07BA007FAB7408F0D083D082D0E03216
:0107C6003200
:0107C70032FF
:0E07C800C0E0C082C0835391EF907FA97402FD
:0807D600F0D083D082D0E032A4
:0807DE00AA82BA81030208ADF2
:0607E600BA82030208B113
:0607EC00BA83030208B508
:0607F200BA84030208B9FD
:0607F800BA85030208BDF2
:0607FE00BA86030208C1E7
:06080400BA87030208C5DB
:06080A00BA88030208C9D0
:06081000BA89030208CDC5
:06081600BA8A030208D1BA
:06081C00BA8B030208D5AF
:06082200BA8C030208D9A4
:06082800BA8D030208DD99
:06082E00BA8E030208E18E
:06083400BA8F030208E583
:06083A00BA91030208E977
:06084000BA92030208ED6C
:06084600BA98030208F15C
:06084C00BA99030208F551
:06085200BAA8030208F938
:06085800BAB8030208FD1E
:06085E00BAC0030209010B
:06086400BAC10302090500
:06086A00BAC803020909EF
:06087000BACA0302090DE3
:06087600BACB03020911D8
:06087C00BACC03020915CD
:06088200BACD03020919C2
:06088800BAD00302091DB5
:06088E00BAD803020921A3
:06089400BAE00302092591
:06089A00BAE8030209297F
:0608A000BAF00302092D6D
:0608A600BAF8030209315B
:0108AC002229
:0408AD00856B8122B4
:0408B100856B8222AF
:0408B500856B8322AA
:0408B900856B8422A5
:0408BD00856B8522A0
:0408C100856B86229B
:0408C500856B872296
:0408C900856B882291
:0408CD00856B89228C
:0408D100856B8A2287
:0408D500856B8B2282
:0408D900856B8C227D
:0408DD00856B8D2278
:0408E100856B8E2273
:0408E500856B8F226E
:0408E900856B912268
:0408ED00856B922263
:0408F100856B982259
:0408F500856B992254
:0408F900856BA82241
:0408FD00856BB8222D
:04090100856BC02220
:04090500856BC1221B
:04090900856BC82210
:04090D00856BCA220A
:04091100856BCB2205
:04091500856BCC2200
:04091900856BCD22FB
:04091D00856BD022F4
:04092100856BD822E8
:04092500856BE022DC
:04092900856BE822D0
:04092D00856BF022C4
:04093100856BF822B8
:08093500AA82BA8103020A063E
:06093D00BA8203020A0B5E
:06094300BA8303020A1052
:06094900BA8403020A1546
:06094F00BA8503020A1A3A
:06095500BA8603020A1F2E
:06095B00BA8703020A2422
:06096100BA8803020A2916
:06096700BA8903020A2E0A
:06096D00BA8A03020A33FE
:06097300BA8B03020A37F3
:06097900BA8C03020A3BE8
:06097F00BA8D03020A3FDD
:06098500BA8E03020A43D2
:06098B00BA8F03020A47C7
:06099100BA9103020A4BBB
:06099700BA9203020A4FB0
:06099D00BA9803020A53A0
:0609A300BA9903020A5795
:0609A900BAA803020A5B7C
:0609AF00BAB803020A5F62
:0609B500BAC003020A6350
:0609BB00BAC103020A6745
:0609C100BAC803020A6B34
:0609C700BACA03020A6F28
:0609CD00BACB03020A731D
:0609D300BACC03020A7712
:0609D900BACD03020A7B07
:0609DF00BAD003020A7FFA
:0609E500BAD803020A83E8
:0609EB00BAE003020A87D6
:0609F100BAE803020A8BC4
:0609F700BAF003020A8FB2
:0609FD00BAF803020A93A0
:030A0300020A974D
:050A0600AA81020A991B
:050A0B00AA82020A9915
:050A1000AA83020A990F
:050A1500AA84020A9909
:050A1A00AA85020A9903
:050A1F00AA86020A99FD
:050A2400AA87020A99F7
:050A2900AA88020A99F1
:050A2E00AA89020A99EB
:040A3300AA8A8062A9
:040A3700AA8B805EA8
:040A3B00AA8C805AA7
:040A3F00AA8D8056A6
:040A4300AA8E8052A5
:040A4700AA8F804EA4
:040A4B00AA91804AA2
:040A4F00AA928046A1
:040A5300AA9880429B
:040A5700AA99803E9A
:040A5B00AAA8803A8B
:040A5F00AAB880367B
:040A6300AAC0803273
:040A6700AAC1802E72
:040A6B00AAC8802A6B
:040A6F00AACA802669
:040A7300AACB802268
:040A7700AACC801E67
:040A7B00AACD801A66
:040A7F00AAD0801663
:040A8300AAD880125B
:040A8700AAE0800E53
:040A8B00AAE8800A4B
:040A8F00AAF0800643
:040A9300AAF880023B
:020A97007A00E3
:030A99008A82222C
:0E0A9C00C0E0C0F0C082C083C002C003C0042E
:0E0AAA00C005C006C007C000C001C0D075D096
:050AB800007A007B0044
:0D0ABD00907FC7E0FCC3EB9C4003020BB62A
:0A0ACA00EB2440F582E4347EF5834E
:090AD400E0FC24FC5003020BB20B
:070ADD00EC2C2C900AE473DD
:070AE400020AF0020B1B02E5
:050AEB000B54020B8119
:0A0AF0000BEB2440F582E4347EF5A0
:0B0AFA0083E0FC0BEB2440F582E434A9
:0A0B05007EF583E0F56B8C82C002E0
:0C0B0F00C0031207DED003D0020B80A24E
:0A0B1B008A040AEC2480FCE4347E16
:0A0B2500FD0BEB2440F582E4347E62
:0E0B2F00F583E0FEF582C002C003C004C005DD
:0E0B3D00120935AE82D005D004D003D0028C50
:090B4B00828D83EEF00B020ABD5D
:0A0B54000BEB2440F582E4347EF53B
:0E0B5E0083E0FC7D00747F2DFD8C068D070B5F
:0A0B6C00EB2440F582E4347EF583AB
:0B0B7600E0F88E828F83F00B020ABDB6
:0A0B81000BEB2440F582E4347EF50E
:0E0B8B0083E0FE7F00747F2FFF8E048F058AAB
:0A0B9900060AEE2480FEE4347EFF1D
:0D0BA3008C828D83E0FC8E828F83F00B022C
:020BB0000ABD7C
:040BB2000B020ABD6B
:050BB600BA00028005F9
:050BBB00907FB7EAF095
:0E0BC000907FC7E4F05391EF907FAA7402F08B
:0E0BCE00D0D0D001D000D007D006D005D00482
:0D0BDC00D003D002D083D082D0F0D0E03220
:0E0BE900C0E0C082C0835391EF907FA97404D6
:080BF700F0D083D082D0E0327F
:0E0BFF00C0E0C082C083907FC9E4F05391EF44
:0D0C0D00907FAA7404F0D083D082D0E03232
:0E0C1A00C0E0C082C0835391EF907FA97408A0
:080C2800F0D083D082D0E0324D
:0E0C3000C0E0C082C083907FCBE4F05391EF10
:0D0C3E00907FAA7408F0D083D082D0E032FD
:0E0C4B00C0E0C082C0835391EF907FA9741067
:080C5900F0D083D082D0E0321C
:0E0C6100C0E0C082C083907FCDE4F05391EFDD
:0D0C6F00907FAA7410F0D083D082D0E032C4
:0E0C7C00C0E0C082C0835391EF907FA9742026
:080C8A00F0D083D082D0E032EB
:0E0C9200C0E0C082C083907FCFE4F05391EFAA
:0D0CA000907FAA7420F0D083D082D0E03283
:0E0CAD00C0E0C082C0835391EF907FA97440D5
:080CBB00F0D083D082D0E032BA
:0E0CC300C0E0C082C083907FD1E4F05391EF77
:0D0CD100907FAA7440F0D083D082D0E03232
:0E0CDE00C0E0C082C0835391EF907FA9748064
:080CEC00F0D083D082D0E03289
:0E0CF400C0E0C082C083907FD3E4F05391EF44
:0D0D0200907FAA7480F0D083D082D0E032C0
:0E0D0F00907F93E0FA54CFF0907F9CE0FA447E
:030D1D0030F02291
:090D2000907F96E0FA4410F022E5
:090D2900907F96E0FA54EFF022ED
:0B0D3200907F96E0FA30E403020D29E8
:030D3D00020D2084
:090D4000907F96E0FA4420F022B5
:090D4900907F96E0FA54DFF022DD
:0B0D5200907F96E0FA30E503020D49A7
:030D5D00020D4044
:07013F00E4F527F528E4F5C3
:0401460023F524F584
:03014A0025F52672
:0A0D6000E521258AFA8A8AC3EA9584
:0A0D6A0021500974012522258CF5A3
:020D74008C22CF
:070D7600E522258CF58C221B
:0B0D7D00AA82AB838A047D008C218BCE
:020D8800222225
:0E0D8A00C28C538EF75389F0438901758A009D
:0E0D9800758C0090B1E0120D7D120D60D2A995
:030DA600D28C22CA
:0E0DA900C0E0C0F0C082C083C002C003C0041E
:0E0DB700C005C006C007C000C001C0D075D086
:0A0DC50000120D60120F34740A25AD
:050DCF0023F523E435CB
:050DD40024F524E435C4
:050DD90025F525E435BD
:040DDE0026F52605CB
:060DE20027E4B52702051D
:010DE80028E2
:090DE900E527B46404E52860026A
:020DF200800877
:060DF400E4F527F52812CA
:020DFA00166A77
:0E0DFC00D0D0D001D000D007D006D005D00452
:0D0E0A00D003D002D083D082D0F0D0E032EF
:05014D00E4F51EF51FA2
:040E1700AA827B80B0
:0D0E1B00907F97E0FC54EFF0EB5A600A90D6
:090E28007F97E0FC4440F08008D3
:080E3100907F97E0FC54BFF034
:0E0E3900907F97E0FC4410F0EBC313FC8C0399
:0B0E470070D2907F97E0FA4440F02248
:0C0E52007A007B80907F97E0FC54BFF09A
:0E0E5E00907F97E0FC54EFF0907F9AE0FC301C
:050E6C00E503EB42026A
:0E0E7100907F97E0FC4410F0EBC313FC8C0361
:0D0E7F0070DD907F97E0FB4440F08A8222F6
:0E0E8C00907F94E0FA548FF0907F9DE0FA443E
:0E0E9A0050F0907F9EE0FA54FBF0907F95E0C0
:0E0EA800FA54FBF0758238120E177582801214
:020EB6000E1715
:0E0EB800907F9BE0FA20E2F8758238120E1748
:060EC6007582A0120E1758
:0C0ECC00907F9BE0FA20E2F87A007B00A7
:0E0ED800C3EA9408EB64809480502874284A82
:0E0EE600FC8B058C82C002C003120E17D003D5
:0E0EF400D00275820CC002C003120E17D0038C
:090F0200D0020ABA00D00B80CD28
:0D0F0B00758201120E17758238120E1790B4
:0E0F18007F95E0FA4404F0D288D2A8907F972B
:0E0F2600E0FA4410F0907F97E0FA4440F02289
:0C0F3400758238120E17758226020E1707
:0C0F4000758238120E17758202020E171F
:0E0F4C00C0E0C0F0C082C083C002C003C00479
:0E0F5A00C005C006C007C000C001C0D075D0E1
:0D0F680000120F40907FB8E0FA30E1030264
:020F75001073F7
:080F7700AA26907E00EAF0AA10
:070F7F0025907E01EAF0AAB3
:0B0F860024907E02EAF07A047B00ACAD
:0C0F9100237D007E007F00907E03ECF0CA
:040F9D007C007D0057
:0E0FA100C3EC9408ED64809480400302106E4F
:0E0FAF0074484CFE8D078E82C002C003C00441
:0E0FBD00C005120E17D005D004D003D0028A52
:080FCB00068B070ABA00010BB6
:0A0FD300EE2400FEEF347EFFC002A2
:0E0FDD00C003C004C005C006C007120E52A813
:0E0FEB0082D007D006D005D004D003D0028EED
:0E0FF900828F83E8F08A068B070ABA00010B8C
:0A100700EE2400FEEF347EFFC0026D
:0E101100C003C004C005C006C007120E52A8DE
:0E101F0082D007D006D005D004D003D0028EB8
:0E102D00828F83E8F08A068B070ABA00010B57
:0A103B00EE2400FEEF347EFFC00239
:0E104500C003C004C005C006C007120E52A8AA
:0E10530082D007D006D005D004D003D0028E84
:0A106100828F83E8F00CBC00010D43
:03106B00020FA1D0
:05106E00907FB9EAF0DB
:07107300051EE4B51E020595
:01107A001F56
:09107B00E51EB46404E51F6002E7
:021084008008E2
:07108600120D52E4F51EF506
:01108D001F43
:0E108E00D0D0D001D000D007D006D005D004BD
:0D109C00D003D002D083D082D0F0D0E0325B
:07015200756900756A007574
:060159006400E4F565F509
:04015F0066F567F5E5
:010163006833
:0810A90085827385837485F0D4
:0510B10075E4F57AF57D
:0410B6007BF57CF555
:0410BA007DF576F555
:0410BE0077F578F555
:0410C20079AD6EAEE8
:0410C6006FAF708513
:0310CA00717E85AF
:0210CD00727F30
:0510CF00A87EAA7F15B8
:0710D4007E74FFB57E0215DA
:0110DB007F95
:0E10DC00C3E49874808AF063F08095F0504170
:0E10EA008D828E838FF0121988FAA3AD82AE2C
:0A10F80083E4FBFCF8EA2576F576A8
:07110200EB3577F577EC35C2
:0511090078F578E835DF
:04110E0079F579E511
:0411120076257AF5CF
:041116007AE57735CA
:04111A007BF57BE501
:04111E0078357CF5AF
:041122007CE57935BA
:051126007DF57D80A4B1
:0A112B00AA767B007C007D0085732E
:09113500828574838575F0EA12CD
:05113E001817AA6BABBD
:041143006CAC6DAD76
:0C1147007A7E007F0078008A828B838C07
:05115300F0ED02181789
:0A115800AA82AB83ACF0AD6BAE6C65
:091162008D078E001DBDFF011E6A
:0E116B00C3E49F748088F063F08095F0501FFD
:0E1179008A828B838CF0121988F5C1A3AA829A
:06118700AB837FA8780293
:05118D001FBFFF011867
:06119200EF4870F780CA6F
:011198002234
:071199007529B5752A627586
:0611A0002B06752C0875FA
:0611A6002D06752E0075F8
:0611AC002FFA75300075FA
:0611B200310175320075E9
:0611B800330075340075E0
:0311BE006B367518
:0611C1006C00756D407525
:0311C7006E2B7517
:0611CA006F007570407516
:0611D000710AE4F57290C3
:0911D600003575F0401210A975F6
:0611DF006B0EE4F56C90BC
:0811E500002975F040021158C9
:0711ED007537B57538627516
:0611F4003906753A07758B
:0611FA003B14753C00757A
:061200003D40753E427501
:061206003F0F754000756A
:06120C0041E87542037584
:0612120043007544007565
:061218004501754600755A
:06121E0047007548007551
:061224004932754A007515
:06122A004B34754C037506
:061230004D00754E007533
:061236004F007550007529
:03123C006B52757D
:06123F006C00756D4075A6
:031245006E39758A
:061248006F007570407597
:06124E007118E4F5729036
:09125400005175F0401210A9755B
:06125D006B1CE4F56C902F
:08126300003775F0400211583C
:09126B00AA827556B5755762752B
:06127400580675590175D2
:06127A005A06755B008AB4
:031280005C855337
:051283005D755E0085B1
:03128800545F852B
:03128B0055607536
:04128E006100756B1B
:0512920063756C00759E
:041297006D40756EC3
:05129B0058756F00759D
:0712A000704075710AE4F5CE
:0812A7007290006275F0401224
:0712AF0010A9756B0EE4F5B8
:0812B6006C90005675F0400237
:0212BE001158C5
:0E12C000907F95E0FA4403F075CDFF75CBFFEB
:0D12CE0075CCEC75CAEC75C834439853908C
:0E12DB007F94E0FA440CF0D2DF758DD9758B4C
:0E12E900D9438E1053890F438920D28E43C003
:0812F700531211991211ED755B
:0612FF0053017554007557
:09130500550075820112126B758E
:06130E0053117554007537
:09131400550075820112126B757F
:06131D0053207554007519
:09132300550075820112126B7570
:06132C0053217554007509
:09133200550075820112126B7561
:06133B00532275540075F9
:09134100550075820112126B7552
:06134A00531075540075FC
:09135000550175820212126B7541
:06135900531175540075EC
:09135F00550175820212126B9017
:0E1368007F95E0FA4408F0D28AD2BCD2ACD213
:04137600BAD2AA221B
:0E137A00C0E0C0F0C082C083C002C003C00447
:0E138800C005C006C007C000C001C0D075D0AF
:0913960000120D32E5646052758D
:06139F006BE8756C03759C
:0613A5006D00756E00856D
:0613AB0065828566838562
:0513B10067F0E5681281
:0E13B600189EAA82AB83ACF0FD0ABA00090BA8
:0813C400BB00050CBC00010D8B
:0713CC00756BE8756C0375F9
:0A13D3006D00756E008A828B838C1A
:0A13DD00F0ED12183085822385839D
:0513E7002485F025F54E
:0413EC0026756400FE
:0E13F000D0D0D001D000D007D006D005D00458
:0D13FE00D003D002D083D082D0F0D0E032F6
:0E140B00C0E0C0F0C082C083C002C003C004B5
:0E141900C005C006C007C000C001C0D075D01D
:0614270000109902800094
:06142D0020980302153AAD
:0B143300AA99C298BAB506756A0102BA
:02143E00150F88
:07144000E56A700302150FBD
:07144700E56AB40102800E0A
:07144E00E56AB402028018F8
:07145500E56AB403348022B4
:0A145C00BA62077401256AFB8002E2
:021466007B0009
:051468008B6A02150F64
:0A146D00BA02077401256AFB800231
:021477007B00F8
:051479008B6A02150F53
:05147E00BA1002800617
:06148300756A0002150F5E
:05148900056A02150FC9
:08148E00056AE56AB4070302D8
:0214960015043B
:07149800E56AB40802800CB4
:07149F00E56AB409028005B3
:0514A600E56AB40A64D0
:0C14AB008A037C007D007E00AF6A7800A0
:0E14B700EF24F9FFE834FFF8C40354F8CFC463
:0E14C50003CF6FCF54F8CF6FF88FF005F08093
:0114D3000C0C
:0C14D400EB2BFBEC33FCED33FDEE33FEA4
:0A14E000D5F0F1EB2565F565EC355C
:0514EA0066F566ED351A
:0514EF0067F567EE3512
:0414F40068F568E54A
:0814F8006AB40A137564017562
:041500006A00800BF2
:061504008A6575660075A2
:05150A00670075680098
:0B150F00907FBCE0FB20E120AB6905F1
:08151A0069EB2400F582E434C2
:0A1522007DF583EAF0E569B4400EA0
:07152C00907FBDE569F07539
:0415330069008003C8
:03153700120D3260
:0E153A00D0D0D001D000D007D006D005D0040C
:0D154800D003D002D083D082D0F0D0E032AA
:0A155500C0D075D00010C102800064
:05155F00A2C0D0D03253
:0E156400907F94E0FA547CF0907F9DE0FA4472
:0E15720083F0907F97E054FEF0E0FA4402F020
:011580002248
:0D158100AA827B047C007D087E007F009024
:0E158E007F97E04401F0E0F854FDF0907F9D5F
:0E159C00E0F84480F0907F97E0F84480F090F3
:0715AA007F97E0F84402F016
:0D15B100907F97E0F854FDF0EB5A600A902F
:0915BE007F97E0F84480F08008FA
:0815C700907F97E0F8547FF0DB
:0E15CF00907F97E0F84402F0EBC313F8880316
:0E15DD0070D2907F97E0FA547FF0907F97E0F5
:0D15EB00FA54FEF0907F97E0FA54FDF09066
:0E15F8007F97E04402F0E054FDF0E0FA440278
:0E160600F0907F97E054FDF0E04402F0E0FA2F
:0B16140054FDF0907F9DE0FA547FF041
:0E161F00907F9AE0FA30E706EC4206ED4207B3
:0E162D00907F97E04402F0E0FA54FDF08C024A
:0E163B00EDC313CA13CAFB8A048B05EA4B7079
:0E164900D5907F97E0FA4402F08E828F8322C4
:0E165700907F95E0FA54EFF0907F9EE0FA4409
:0516650010F002156405
:0D166A00907F98E04410F0E0FA54EFF02279
:0E1677001201000100000040470502100100B2
:04168500010200015D
:0916890009023C00010100A0006F
:091692000904000006FF0000003D
:07169B0007050102400000F9
:0716A20007050202400000F1
:0716A90007050402400000E8
:0716B0000705810240000064
:0716B700070582024000005C
:0716BE000705840240000053
:0416C500040309040D
:0A16C9000A035200470049004F00D9
:0A16D3000A03560031003000300019
:0216DD0000000B
:03004300021B009D
:091B000002073500020763000230
:081B0900074D000207AE0002C7
:081B11000779000207AD000294
:081B190007C6000207C7000225
:081B210007C800020A9C000243
:081B29000BE900020BFF0002B2
:081B31000C1A00020C30000246
:081B39000C4B00020C610002DC
:081B41000C7C00020C92000272
:081B49000CAD00020CC3000208
:071B51000CDE00020CF400A1
:0816DF00FB7A20E4FCFDFEFF94
:0E16E700E5822582F582E58333F583E5F03355
:0B16F500F5F0EB33FB4017DAE9804210
:0E170000E5822582F582E58333F583E5F0333B
:05170E00F5F0EB33FBD8
:0E171300EC33FCED33FDEE33FEEF33FFEC95CF
:061721006BED956CEE95E6
:081727006DEF956E4013EC9587
:08172F006BFCED956CFDEE95DD
:091737006DFEEF956EFF43820187
:02174000DABE0F
:02174200EB2298
:0E174400907FD6E04408F0E054FBF0E0FA4459
:0517520008F03004085E
:08175700907FD6E0FA4402F095
:0E175F009005DC12193B907F92E0FA30E30611
:06176D009005DC12193B9F
:0D177300907FAB74FFF0907FA974FFF090A1
:0E1780007FAA74FFF05391EF907FD6E054F7EC
:06178E00F0E0FA4404F053
:011794002232
:06011500E478FFF6D8FDBE
:08179500AA82AB0AAC0B7D0037
:0E179D0074012BF582E43CF583E0FEBE026889
:0717AB008D060DEEB50205ED
:0517B2008B828C8322F4
:0D17B70074022BF582E43CF583E0F56BA392
:0617C400E0F56CAE6B9035
:0C17CA00006C75F000121988FF62068E9A
:0817D6006B90006C75F000122D
:0917DE001988FEE56BFF6206901C
:0A17E700006C75F000EE121817AE4A
:0817F1006B90006C75F0001212
:0C17F9001988FF62068E6B8B068C07E5DA
:0C1805006B2EFEE56C3FFF8E038F04028B
:02181100179D21
:0318130090000042
:0118160022AF
:0800F3007900E94400601B7A6A
:0500FB00009019B97826
:030100000075A0E7
:0A01030000E493F2A308B80002051F
:08010D00A0D9F4DAF275A0FF9D
:0E18170020F71030F6118883A88220F507F61E
:05182500A8837583009B
:01182A00229B
:03182B00F280F751
:02182E00F022A6
:0C183000AAF0FBE582856BF0A4FCADF093
:0C183C00E583856BF0A42DFDE435F0FE83
:0C184800E582856CF0A42DFDE5F03EFE6D
:0C185400E433FFEA856BF0A42EFEE5F003
:0C1860003FFFE583856CF0A42EFEE5F050
:0C186C003FFFE582856DF0A42EFEE5F044
:0B1878003FFFEB856BF0A42FFFEA851B
:0A1883006CF0A42FFFE583856DF0E3
:0C188D00A42FFFE582856EF0A42F8EF0E2
:051899008D838C82220A
:08011B007800E84400600A7955
:030123000075A0C4
:0601260000E4F309D8FC1F
:08012C007800E84400600C7942
:0B01340000900000E4F0A3D8FCD9FA12
:0E189E00FBC2D530E715D2D5E4C39582F582A2
:0D18AC00E49583F583E495F0F5F0E49BFBF3
:0A18B900E56E30E717B2D5E4C395E1
:0518C3006BF56BE495DC
:0518C8006CF56CE495D5
:0518CD006DF56DE495CE
:0318D2006EF56E42
:0E18D500EB1216DF30D513FBE4C39582F582CB
:0C18E300E49583F583E495F0F5F0E49BB8
:0118EF0022D6
:0618F000AA82AB0CAC0D56
:0E18F60074012BF582E43CF583E0FDBD032375
:061904008A051AED7005D2
:05190A008B828C83229A
:0E190F008B058C068B828C83E0FF7800EF2D19
:0A191D00FDE83EFE8D038E0480CF2E
:031927009000002D
:01192A00229A
:0E192B00907FD6E04480F0438701000000006A
:0219390000228A
:0C193B00AA82AB83907F92E0FC30E307AF
:07194700EBCA25E0CA33FBE7
:09194E008A048B051ABAFF011B83
:04195700EC4D600DE6
:0D195B00C002C0031219A4D003D00280E620
:01196800225C
:08196900907FD6E0FA30E7168A
:0E197100907FD6E0FA4401F090001412193B6A
:08197F00907FD6E0FA54FEF05F
:01198700223D
:0300E60075817FA2
:0A00E9001219B5E5826003020167F9
:0E19880020F71430F6148883A88220F507E6B5
:06199600A8837583002206
:03199C00E280F7EF
:03199F00E49322AC
:0219A200E02241
:0919A4007400F58690FDA57C0598
:0819AD00A3E582458370F922D5
:0419B5007582002215
:00000001FF
